:020000040000FA
:100000002EEF29F01200120072EF02F01200010030
:10001000C052000000010000F90000000F0E93160E
:100020008116939493968194819600D90F0E811630
:10003000300E811227D81FD90F0E8116300E811273
:1000400021D819D90F0E8116300E81121BD813D961
:100050000F0E8116818A16D8280EE66E17D8E55243
:10006000080EE66E13D8E552010EE66E0FD8E55283
:10007000060EE66E0BD8E5520C0EE66E07D8E5527A
:1000800000D0120081861CD981961200D9CFE6FFDC
:10009000E1CFD9FF1AD9819481960F0E8116FE0EF9
:1000A000DB50F00B8112EEDF0F0E8116FE0EDB38F7
:1000B000F00BF00B8112E6DF00D0E552E7CFD9FF5D
:1000C0001200D9CFE6FFE1CFD9FFFFD88184819616
:1000D0000F0E8116FE0EDB50F00B81128186F0D8D8
:1000E00081960F0E8116FE0EDB38F00BF00B81129D
:1000F0008186E6D8819600D0E552E7CFD9FF12007D
:10010000D9CFE6FFE1CFD9FFFD0EDBCFF6FFFE0E24
:10011000DBCFF7FF0800F55011E0FD0EDBCFF6FF57
:10012000FE0EDBCFF7FF0800F550E66ECADFE552A2
:10013000FD0EDB2AFE0E01E3DB2AE6D700D0E552F6
:10014000E7CFD9FF1200D9CFE6FFE1CFD9FFFD0EEF
:10015000DBCFE9FFFE0EDBCFEAFFEF5010E0FD0E34
:10016000DBCFE9FFFE0EDBCFEAFFEF50E66EA9DF43
:10017000E552FD0EDB2AFE0E01E3DB2AE8D700D0B4
:10018000E552E7CFD9FF1200D9CFE6FFE1CFD9FF83
:10019000E652FE0EDB0404E1FD0EDB50800FDF6E45
:1001A000FE0EDB50020804E1FD0EDB50C00FDF6ED7
:1001B000DFCFE6FF6BDFE552E552E552E7CFD9FF2F
:1001C0001200D9CFE6FFE1CFD9FF020EE126E66AA1
:1001D000FE0EDBCFE6FFD8DFE552E552DE6ADD6AD0
:1001E000DECF14F0DDCF15F0D890155004E6100ED8
:1001F000145C000E155809E2200EE66E62DFE5522F
:10020000DF2A010E01E3DB2AEBD7E66AFE0EDBCF25
:10021000E6FFBADFE552E552020EE15C02E2E16A76
:10022000E552E16EE552E7CFD9FF1200D9CFE6FFE4
:10023000E1CFD9FF020EE126DE6ADD6ADECF14F0DF
:10024000DDCF15F0D890155004E6100E145C270E83
:10025000155806E20000DF2A010E01E3DB2AEED783
:1002600000D0020EE15C02E2E16AE552E16EE55285
:10027000E7CFD9FF1200D9CFE6FFE1CFD9FF020EB9
:10028000E126DE6ADD6ADECF14F0DDCF15F0D8900E
:10029000155004E6C40E145C090E155806E2000061
:1002A000DF2A010E01E3DB2AEED700D0020EE15C6B
:1002B00002E2E16AE552E16EE552E7CFD9FF1200B2
:1002C00000000000000000001200D9CFE6FFE1CFDF
:1002D000D9FF020EE126DE6ADD6ADECF14F0DDCF43
:1002E00015F0D890155004E6E80E145C030E15586E
:1002F00006E20000DF2A010E01E3DB2AEED700D080
:10030000020EE15C02E2E16AE552E16EE552E7CFFE
:10031000D9FF1200D9CFE6FFE1CFD9FF81940F0EAC
:100320008116FE0EDB504009F00B8112C9DFAADEF8
:100330000F0E8116FE0EDB38F00BF00B8112C0DFC2
:10034000A1DE00D0E552E7CFD9FF12000000000087
:10035000000000000000000000000000000000009D
:10036000000000001200400EE66EE66A740EE66EB3
:1003700028EC28F0E552E552E5529F8AD08E9D9AEE
:10038000F29CF29E1200D9CFE6FFE1CFD9FF020E18
:10039000E126DE6ADD6AFD0EDBCFF6FFFE0EDBCF67
:1003A000F7FF0800F55015E0FD0EDBCFF6FFFE0E5F
:1003B000DBCFF7FF0800F550E66E55D8E552DF2A8F
:1003C000010E01E3DB2AFD0EDB2AFE0E01E3DB2A30
:1003D000E2D7DECF14F0DDCF15F014C0F3FF15C067
:1003E000F4FF020EE15C03E200D0E16AE552E16E47
:1003F000E552E7CFD9FF1200D9CFE6FFE1CFD9FF11
:10040000020EE126DE6ADD6AFD0EDBCFE9FFFE0E9D
:10041000DBCFEAFFEF5014E0FD0EDBCFE9FFFE0E6D
:10042000DBCFEAFFEF50E66E1ED8E552DF2A010E61
:1004300001E3DB2AFD0EDB2AFE0E01E3DB2AE4D713
:10044000DECF14F0DDCF15F014C0F3FF15C0F4FFBC
:10045000020EE15C03E200D0E16AE552E16EE55292
:10046000E7CFD9FF1200D9CFE6FFE1CFD9FFACA289
:10047000FED7FE0EDBCFE6FFDFEC28F0E552E552BB
:10048000E7CFD9FF12000D0EE66EEDDFE5520A0E42
:10049000E66EE9DFE5521200D9CFE6FFE1CFD9FFE2
:1004A000E65207010451021902E10551031901E165
:1004B000F8D702C7E9FF03C7EAFF022B000E0323A8
:1004C000EFCFDFFFA00E025D000E035904E3600EC4
:1004D000026F000E036FDF5000D0E552E552E7CF08
:1004E000D9FF1200DACFE4FFE2CFDAFFE9CFE4FF71
:1004F000EACFE4FFF6CFE4FFF7CFE4FFF5CFE4FF68
:10050000F3CFE4FFF4CFE4FFFACFE4FF00EE00F016
:10051000140EE80403E3EECFE4FFFBD700EE14F083
:10052000140EE80403E3EECFE4FFFBD7E6529D5040
:10053000200B30E09E50200B2DE088EC28F00701C6
:10054000136FABA407D0AB9E8B81112B000E12232F
:10055000AB8E01D08B91ABA207D0AB988B83AB88CD
:100560000F2B000E102301D08B93ACA2FED70701F6
:1005700004C7E9FF05C7EAFF042B000E052313C7D4
:10058000EFFFA00E045D000E055904E3600E046F3A
:10059000000E056FF250100B17E0F250020B14E042
:1005A000070113510CE11B0E136F9D9A9E9A600E6A
:1005B000046F000E056F04C702F705C703F7F29238
:1005C000F2989D9A81EC0FF0E55200EE27F0140EA0
:1005D000E80403E3E5CFEDFFFBD700EE13F0140EC4
:1005E000E80403E3E5CFEDFFFBD7E5CFFAFFE5CF66
:1005F000F4FFE5CFF3FFE5CFF5FFE5CFF7FFE5CF5C
:10060000F6FFE5CFEAFFE5CFE9FFE5CFDAFF11001E
:10061000D9CFE6FFE1CFD9FFFF0EE76EFD0EDBCFAE
:1006200014F0FE0EDBCF15F0E7501416156A1450C7
:10063000A96EFD0EDBCF14F0FE0EDBCF15F015C05A
:1006400014F0156A030E1414AA6EA69EA69CA6802A
:10065000E80EE66E030EE66EE66AE66ADCEC09F08A
:10066000E552E552E552E552A85000D0E552E7CFF9
:10067000D9FF1200D9CFE6FFE1CFD9FF020EE12664
:1006800007018AAF11D0E76EFD0EDBCF14F0FE0E2E
:10069000DBCF15F0E7501426000E1522FD0E14C016
:1006A000DBFFFE0E15C0DBFFFD0EDBCF14F0FE0EF0
:1006B000DBCF15F015C014F0156A030E1414AA6EE2
:1006C000FF0EE76EFD0EDBCF14F0FE0EDBCF15F054
:1006D000E7501416156A1450A96EFC0EDB50A86E74
:1006E000A69EA684A69CF2AE04D0F29E010EDE6EFB
:1006F000DD6A550EA76EAA0EA76EA682A1A8FED728
:10070000A198A694D9CFE9FFDACFEAFF010EEE183F
:1007100001E1ED5001E1F28E020EE15C02E2E16ADC
:10072000E552E16EE552E7CFD9FF1200D9CFE6FFDF
:10073000E1CFD9FFFB0EDBCFE9FFFC0EDBCFEAFFF9
:10074000EF5022E0FB0EDBCFE9FFDB2AFC0EDBCF14
:10075000EAFF01E3DB2AEF50E66ED950FD0FE96EA8
:10076000FF0EDA20EA6EEECF14F0EDCF15F0020E98
:10077000EE26000EEF2214C0E6FF15C0E6FF7ADF7A
:10078000E552E552E552D6D7E552E7CFD9FF120040
:10079000D9CFE6FFE1CFD9FF040EE12607018AAFEA
:1007A00017D0FD0EDBCF14F0FE0EDBCF15F0040EDC
:1007B000D89014361536E804FBE1000E1426020E1C
:1007C0001522FD0E14C0DBFFFE0E15C0DBFF12D09C
:1007D000FD0EDBCF14F0FE0EDBCF15F0050ED8902A
:1007E00014361536E804FBE1FD0E14C0DBFFFE0EE7
:1007F00015C0DBFF020EDB6A030EDB6AD950FD0F6A
:10080000E96EFF0EDA20EA6EFF0ED880EE54030E7A
:10081000ED5401E241D0FD0EDBCFE6FFFE0EDBCF53
:10082000E6FFF6DEE552E552DE6EDD6AD9CFE9FF7E
:10083000DACFEAFFEE50ED1001E12ED007018A5128
:10084000800B0EE0020EDBCF14F0030EDBCF15F0B1
:10085000153404E214500F08000E155401E21CD0A8
:100860008ABF05D0DFCFE6FFFEDDE55204D0DFCF43
:10087000E6FF27DCE552FD0EDB2AFE0E01E3DB2A54
:10088000020EDB2A030E01E3DB2AD9CFE9FFDACF20
:10089000EAFFEE50ED10B2E1E80EE66E030EE66EF2
:1008A000E66AE66ADCEC09F0E552E552E552E5520B
:1008B000040EE15C02E2E16AE552E16EE552E7CF47
:1008C000D9FF1200D9CFE6FFE1CFD9FF040EE12610
:1008D0000701E00E006F010E016F00C7E6FF01C7C0
:1008E000E6FFFD0EDBCFE6FFFE0EDBCFE6FF96EC6C
:1008F00023F0E552E552E552E55200C7E6FF01C795
:10090000E6FF7AEC28F0E552E552F3CFDEFFF4CFB4
:10091000DDFFD9CFE9FFDACFEAFF020EEECFDBFF32
:10092000030EEDCFDBFF020EDBCF14F0030EDBCFA7
:1009300015F0040E145C000E155813E207018ABF6F
:1009400005D0300EE66E8FDDE55205D0300EE66E36
:1009500061EC00F0E552020EDB2A030E01E3DB2A14
:10096000E2D707018ABF0CD000C7E6FF01C7E6FF48
:1009700043DDE552E552F3CFDEFFF4CFDDFF08D0D3
:1009800000C7E6FF01C7E6FFA3EC00F0E552E55221
:10099000040EE15C02E2E16AE552E16EE552E7CF66
:1009A000D9FF1200D9CFE6FFE1CFD9FF0E0EE12625
:1009B000F90EDBCFDEFFDBCFDDFFF80EDB500008EA
:1009C00002E3070E08D0F80EDB50160802E2170EFD
:1009D00002D0F80EDB28E66ED950080FE96EDACFA8
:1009E000EAFFE552E750EE6EED6A020EDB6A030E97
:1009F000DB6AFB0EDBCF14F0FC0EDBCF15F0FD0E37
:100A0000DBCF16F0FE0EDBCF17F00C6A0D6A0E6A14
:100A10000F6A14C007F015C008F016C009F017C01F
:100A20000AF0EEEC1EF0010A33E1F90EDBCFE9FF2C
:100A3000DB2AFA0EDBCFEAFF01E3DB2A2D0EEF6E95
:100A4000FB0EDBCF14F0FC0EDBCF15F0FD0EDBCF81
:100A500016F0FE0EDBCF17F00C6A0D6A800E0E6EDC
:100A6000BF0E0F6E14C007F015C008F016C009F0D5
:100A700017C00AF0C5EC1DF0FB0E07C0DBFFFC0E33
:100A800008C0DBFFFD0E09C0DBFFFE0E0AC0DBFF66
:100A9000FB0EDBCF14F0FC0EDBCF15F0FD0EDBCF31
:100AA00016F0FE0EDBCF17F00C6A0D6A0E6A0F6AA5
:100AB00014C007F015C008F016C009F017C00AF0FE
:100AC000E5EC1EF0010A4AE1FB0EDBCF14F0FC0E50
:100AD000DBCF15F0FD0EDBCF16F0FE0EDBCF17F0EF
:100AE0000C6A0D6A800E0E6E3F0E0F6E14C007F07A
:100AF00015C008F016C009F017C00AF0EEEC1EF0A1
:100B0000010A2CE1146A156A200E166E410E176E4A
:100B1000D950FB0FE96EFF0EDA20EA6EEECF07F038
:100B2000EECF08F0EECF09F0EFCF0AF014C00CF0D2
:100B300015C00DF016C00EF017C00FF0C5EC1DF07B
:100B40000AC0EDFF09C0EDFF08C0EDFF07C0EFFFD1
:100B5000020EDB06030E01E2DB06B6D7FB0EDBCF8F
:100B600014F0FC0EDBCF15F0FD0EDBCF16F0FE0E01
:100B7000DBCF17F00C6A0D6A200E0E6E410E0F6E61
:100B800014C007F015C008F016C009F017C00AF02D
:100B9000EEEC1EF0010A2EE0FB0EDBCF14F0FC0E93
:100BA000DBCF15F0FD0EDBCF16F0FE0EDBCF17F01E
:100BB0000C6A0D6A200E0E6E410E0F6E14C007F007
:100BC00015C008F016C009F017C00AF072EC1DF04D
:100BD000FB0E07C0DBFFFC0E08C0DBFFFD0E09C0EB
:100BE000DBFFFE0E0AC0DBFF020EDB2A030E01E371
:100BF000DB2AB4D7020EDBCF14F0030EDBCF15F0E7
:100C0000D950080FE96EDACFEAFF1450EE261550DE
:100C1000ED22010EF36E040EF3CFDBFF050EDB6A4F
:100C2000040EDBCF08F0050EDBCF09F0ADEC1CF0B5
:100C30000A0E07C0DBFF0B0E08C0DBFF0C0E09C05D
:100C4000DBFF0D0E0AC0DBFF040EDBCF14F0050E38
:100C5000DBCF15F0080EDBCF16F0090EDBCF17F057
:100C600015501718E8AE02D0173404D01650145C93
:100C7000175015582EE20A0EDBCF14F00B0EDBCF07
:100C800015F00C0EDBCF16F00D0EDBCF17F00C6A53
:100C90000D6A200E0E6E410E0F6E14C007F015C0C7
:100CA00008F016C009F017C00AF072EC1DF00A0E29
:100CB00007C0DBFF0B0E08C0DBFF0C0E09C0DBFF1B
:100CC0000D0E0AC0DBFF040EDB2A050E01E3DB2A52
:100CD000BBD70A0EDBCF18F00B0EDBCF19F00C0ED2
:100CE000DBCF1AF00D0EDBCF1BF00C6A0D6A0E6A1B
:100CF000400E0F6E18C007F019C008F01AC009F0B6
:100D00001BC00AF072EC1DF007C014F008C015F00B
:100D100009C016F00AC017F0D950FB0FE96EFF0E9C
:100D2000DA20EA6EEECF07F0EECF08F0EECF09F052
:100D3000EFCF0AF014C00CF015C00DF016C00EF085
:100D400017C00FF0DCEC1CF00AC0EDFF09C0EDFF8E
:100D500008C0EDFF07C0EFFFFB0EDBCF14F0FC0E69
:100D6000DBCF15F0FD0EDBCF16F0FE0EDBCF17F05C
:100D70000C6A0D6A200E0E6E410E0F6E14C007F045
:100D800015C008F016C009F017C00AF0EEEC1EF00E
:100D9000010A13E0FB0EDB6AFC0EDB6A800EF36EC9
:100DA000FD0EF3CFDBFF3F0EF36EFE0EF3CFDBFF46
:100DB000020EDB2A030E01E3DB2A020EDBCF14F066
:100DC000030EDBCF15F00001800E15145FE0F90E65
:100DD000DBCFE9FFDB2AFA0EDBCFEAFF01E3DB2AF8
:100DE000300EEF6EF90EDBCFE9FFDB2AFA0EDBCF18
:100DF000EAFF01E3DB2A2E0EEF6E080EDBCF14F0C4
:100E0000090EDBCF15F0800E151414E0020EDBCFB7
:100E100016F0030EDBCF17F0080EDB50165C146ED5
:100E2000090EDB501758156E020E14C0DBFF030EBF
:100E300015C0DBFF040EDB68050EDB68040EDBCF9C
:100E400014F0050EDBCF15F0020EDBCF16F0030E0B
:100E5000DBCF17F017501518E8AE02D0153404D0C8
:100E60001450165C1550175811E2F90EDBCFE9FF4C
:100E7000DB2AFA0EDBCFEAFF01E3DB2A300EEF6E4E
:100E8000040EDB06050E01E2DB06D8D7040EDB6A92
:100E9000050EDB6A040EDBCF14F0050EDBCF15F078
:100EA000080EDBCF16F0090EDBCF17F01550171820
:100EB000E8AE02D0173404D01650145C1750155801
:100EC00001E3ACD0FB0EDBCF07F0FC0EDBCF08F06C
:100ED000FD0EDBCF09F0FE0EDBCF0AF07FEC1EF03B
:100EE000060E08C0DBFF070E09C0DBFF300EE76E01
:100EF000060EDBCF14F0070EDBCF15F0E7501426FB
:100F0000000E1522F90EDBCFE9FFDB2AFA0EDBCF4C
:100F1000EAFF01E3DB2A14C0EFFF040EDBCF14F07D
:100F2000050EDBCF15F0020EDB50141803E1030EA3
:100F3000DB5015180BE1F90EDBCFE9FFDB2AFA0EC7
:100F4000DBCFEAFF01E3DB2A2E0EEF6E060EDBCFCE
:100F500008F0070EDBCF09F0ADEC1CF00A0E07C05D
:100F6000DBFF0B0E08C0DBFF0C0E09C0DBFF0D0E14
:100F70000AC0DBFF07C014F008C015F009C016F066
:100F80000AC017F0D950FB0FE96EFF0EDA20EA6EA7
:100F9000EECF07F0EECF08F0EECF09F0EFCF0AF07A
:100FA00014C00CF015C00DF016C00EF017C00FF0F5
:100FB000DBEC1CF00AC0EDFF09C0EDFF08C0EDFF3F
:100FC00007C0EFFF146A156A200E166E410E176EE9
:100FD000D950FB0FE96EFF0EDA20EA6EEECF07F074
:100FE000EECF08F0EECF09F0EFCF0AF014C00CF00E
:100FF00015C00DF016C00EF017C00FF0C5EC1DF0B7
:101000000AC0EDFF09C0EDFF08C0EDFF07C0EFFF0C
:10101000040EDB2A050E01E3DB2A3CD7F90EDBCFF9
:10102000E9FFFA0EDBCFEAFFEF6A0E0EE15C02E2A7
:10103000E16AE552E16EE552E7CFD9FF1200D9CF60
:10104000E6FFE1CFD9FF060EE12607018A9DFB0EE0
:10105000DBCF07F0FC0EDBCF08F0FD0EDBCF09F095
:10106000FE0EDBCF0AF0AEEC1EF006C0DEFF07C0BE
:10107000DEFF08C0DEFF09C0DDFFDD52DD52F90EE4
:10108000DBCF08F0FA0EDBCF09F0ADEC1CF007C0A7
:1010900014F008C015F009C016F00AC017F0FB0ED6
:1010A000DBCF1CF0FC0EDBCF1DF0FD0EDBCF1EF006
:1010B000FE0EDBCF1FF0D9CFE9FFDACFEAFFEECF8C
:1010C00024F0EECF25F0EECF26F0EFCF27F024C0AE
:1010D00006F025C007F026C008F027C009F0C2ECD2
:1010E0001CF007C020F008C021F009C022F00AC09F
:1010F00023F020C00CF021C00DF022C00EF023C060
:101100000FF01CC007F01DC008F01EC009F01FC082
:101110000AF0DBEC1CF007C018F008C019F009C099
:101120001AF00AC01BF018C00CF019C00DF01AC05C
:101130000EF01BC00FF014C007F015C008F016C069
:1011400009F017C00AF0C5EC1DF07FEC1EF0040E8C
:1011500008C0DBFF050E09C0DBFF9E0EE66E010E28
:10116000E66ED9CFE9FFDACFEAFFEECFE6FFEECFAA
:10117000E6FFEECFE6FFEFCFE6FF30EC24F0146E93
:10118000060EE15E145007018AAF09D09E0EE66E8E
:10119000010EE66EA3EC00F0E552E5520CD09E0E77
:1011A000E66E010EE66EFCEC01F0E552E552F3CF7F
:1011B00018F7F4CF19F707018AAF06D02E0EE66EA6
:1011C00061EC00F0E55205D02E0EE66E33EC02F035
:1011D000E552040EDBCFE6FF050EDBCFE6FF62EC47
:1011E00004F0E552E552060EE15C02E2E16AE552E6
:1011F000E16EE552E7CFD9FF12000F01426B428F3B
:10120000429B428907011A510F01030BF36EF3460B
:10121000F346F346F346CF0E4215F310426F1AC75A
:1012200014F01BC715F0030ED89014361536E806D7
:10123000FBE1B60E1426450E1522166A14C0E6FF11
:1012400015C0E6FF16C0E6FF9E0EE66E010EE66EC6
:1012500061EC28F0176E050EE15E175007018AAFAA
:101260000ED0020EE66EE1EC00F0E5529E0EE66E48
:10127000010EE66EA3EC00F0E552E5520ED09E0E94
:10128000E66E010EE66EFCEC01F0E552E552F3CF9E
:1012900018F7F4CF19F743EC02F0E80EE66E030EF0
:1012A000E66EE66AE66A88D8E552E552E552E5520E
:1012B0000F01418F419D418B41874195419541915E
:1012C000406B1200D9CFE6FFE1CFD9FFE652800E86
:1012D000DF6EDF50000813E2FE0EDB50DF1406E085
:1012E000310EE66E33EC02F0E55205D0300EE66EBC
:1012F00033EC02F0E552DF407F0BDF6EEAD7E552B8
:10130000E552E7CFD9FF1200D9CFE6FFE1CFD9FFF1
:10131000020EE126010EDB6AFE0EDB50F00BE83810
:101320000F0B300FDF6EDF50390803E2070EDF24AA
:10133000DF6EFE0EDB500F0B300FE76E010EE7CFB6
:10134000DBFFDB5039080AE2070E146E010EDBCF1B
:10135000E7FF1450E726010EE7CFDBFF07018ABF46
:1013600011D0DFCFE6FF33EC02F0E552010EDBCF08
:10137000E6FF33EC02F0E552680EE66E33EC02F065
:10138000E55210D0DFCFE6FF61EC00F0E552010E30
:10139000DBCFE6FF61EC00F0E552680EE66E61EC33
:1013A00000F0E552020EE15C02E2E16AE552E16E14
:1013B000E552E7CFD9FF1200D9CFE6FFE1CFD9FF41
:1013C000FB0EDBCF07F0FC0EDBCF08F0FD0EDBCF12
:1013D00009F0FE0EDBCF0AF00A34000E0A1809E607
:1013E000D880000E0754000E0854000E0954000E59
:1013F0000A540CE2D950FB0FE96EFF0EDA20EA6EB8
:10140000EE06000EEE5AEE5AEE5ADAD7E552E7CF64
:10141000D9FF1200D9CFE6FFE1CFD9FF020EE126B6
:10142000DE6ADD6ADECF14F0DDCF15F0FE0EDB5094
:10143000000115AE02D0D89003D0145C000E1558F0
:101440000AE2200EE66E33EC02F0E552DF2A010ECE
:1014500001E3DB2AE7D7020EE15C02E2E16AE55232
:10146000E16EE552E7CFD9FF12008168010E936E5D
:101470000F01396B070E806E386B38813883926E9E
:10148000806A82683A6B9F0E946E948E949C606A18
:101490001200C280C19EC08EC08AC088C096C08221
:1014A000C094C090C196C194C192C1901200D9CF8E
:1014B000E6FFE1CFD9FF040EE126FD0EDBCF14F0ED
:1014C000FE0EDBCF15F0D89014361536D8901436B2
:1014D0001536010E1424C26E0A0EE66E3CEC29F09D
:1014E000E5525EEC29F059EC29F0000901E0FBD748
:1014F00047EC29F0F3CFDEFFF4CFDDFFDECF14F0B1
:10150000DDCF15F014C0F3FF15C0F4FF040EE15C4D
:1015100003E200D0E16AE552E16EE552E7CFD9FF80
:101520001200CD9ECD9CCD8ACD88CD96CD94CD8216
:10153000CD90CC9ECC9ACC92CC909F80D08EDB0E5E
:10154000E66E0B0EE66EA7EC28F0E552E5529E9093
:10155000F29CCD909D90F29EF29C1200D9CFE6FFB6
:10156000E1CFD9FF020EE126DE6ADD6AFB0EDBCF9A
:10157000F6FFDB2AFC0EDBCFF7FF01E3DB2A0800D6
:10158000F550E66EFD0EDBCFE9FFDB2AFE0EDBCF6A
:10159000EAFF01E3DB2AE552E750EF6EDF2A010E96
:1015A00001E3DB2ADECF14F0DDCF15F0D890155023
:1015B00004E6000E145C010E1558D8E3020EE15C3F
:1015C00002E2E16AE552E16EE552E7CFD9FF12008F
:1015D000D9CFE6FFE1CFD9FF020EE126DE6ADD6A50
:1015E000FB0EDBCFF6FFDB2AFC0EDBCFF7FF01E3C0
:1015F000DB2A0800F550E66EFF0EE76EFD0EDBCF2E
:1016000014F0FE0EDBCF15F0E7501426000E152265
:10161000DE50145CE96EDD501558EA6EE552E75075
:10162000EF6EDF2A010E01E3DB2ADECF14F0DDCFFF
:1016300015F0D890155004E6000E145C010E1558F4
:10164000CFE3020EE15C02E2E16AE552E16EE552AF
:10165000E7CFD9FF1200D9CFE6FFE1CFD9FFFB0ECC
:10166000DBCF14F0FC0EDBCF15F0FD0EDBCF16F058
:10167000FE0EDBCF17F014C006F015C007F016C041
:1016800008F017C009F0C2EC1CF007C068F708C0EA
:1016900069F709C06AF70AC06BF7240EF66E440EAC
:1016A000F76E0900F5CF6CF70900F5CF6DF709006B
:1016B000F5CF6EF70800F5CF6FF76CC70CF06DC76C
:1016C0000DF06EC70EF06FC70FF068C707F069C75F
:1016D00008F06AC709F06BC70AF072EC1DF007C08A
:1016E00064F708C065F709C066F70AC067F764C702
:1016F000E6FF65C7E6FF66C7E6FF67C7E6FF51EC92
:1017000027F0E552E552E552E55206C014F007C055
:1017100015F008C016F009C017F014C007F015C086
:1017200008F016C009F017C00AF0AEEC1EF006C0B3
:1017300082F707C083F708C084F709C085F707015F
:101740008A8F020EE66EE1EC00F0E5520701090E09
:10175000781901E1795140E120C714F021C715F053
:101760000A0E0D6E0E6A14C008F015C009F032ECB6
:101770001EF008C014F009C015F0300E1424E66EF7
:1017800061EC00F0E55220C714F021C715F00A0EF5
:101790000D6E0E6A14C008F015C009F032EC1EF090
:1017A00004C014F005C015F0300E1424E66E61EC90
:1017B00000F0E552200EE66E61EC00F0E552200EDE
:1017C000E66E61EC00F0E552060EE66E020EE66E85
:1017D000C4EC00F0E552E552010EE66EDEC1E6FF14
:1017E000DFC1E6FF68C7E6FF69C7E6FF6AC7E6FF35
:1017F0006BC7E6FFD2EC04F0146E070EE15E1450E6
:10180000DEC1E6FFDFC1E6FFA3EC00F0E552E552E2
:10181000200EE66E61EC00F0E552480EE66E61ECDB
:1018200000F0E5527A0EE66E61EC00F0E552070139
:101830008A9FDEC1E6FFDFC1E6FFFCEC01F0E55266
:10184000E552F3CF18F7F4CF19F7480EE66E33ECF4
:1018500002F0E5527A0EE66E33EC02F0E55243EC0C
:1018600002F007018A8F82C797F783C796F784C76C
:1018700095F7866B876B886B896BE552E7CFD9FF4D
:1018800012000701600E046F000E056F04C702F717
:1018900005C703F78E6B8F6B136B076B1200070185
:1018A000010E0B1901E10C5109E18250E66E0ADDCF
:1018B000E552090EE66E33EC02F0E5520701A06B2B
:1018C000A16B82B02AD0500EE66EC30EE66EE66AB9
:1018D000E66A72DDE552E552E552E55282B01DD06E
:1018E0000701782B000E7923793504E278510A0834
:1018F000000E795503E2010E786F796B500EE66E9B
:10190000C30EE66EE66AE66A57DDE552E552E55239
:10191000E552010E0701A06FA16B0701A13504E29A
:10192000A0510008000EA15505E2A0C7F3FFA1C712
:10193000F4FFAED082B226D0500EE66EC30EE66E35
:10194000E66AE66A39DDE552E552E552E55282B2D1
:1019500019D007017807000E795B7851791103E1FE
:101960000A0E786F796B500EE66EC30EE66EE66A6D
:10197000E66A22DDE552E552E552E552020E070124
:10198000A06FA16B0701A13504E2A0510008000E71
:10199000A15505E2A0C7F3FFA1C7F4FF79D082B833
:1019A0001CD0500EE66EC30EE66EE66AE66A04DDF3
:1019B000E552E552E552E55282B80FD0500EE66E80
:1019C000C30EE66EE66AE66AF7DCE552E552E552DA
:1019D000E552030E0701A06FA16B0701A13504E2D8
:1019E000A0510008000EA15505E2A0C7F3FFA1C752
:1019F000F4FF4ED082B41CD0500EE66EC30EE66EDD
:101A0000E66AE66AD9DCE552E552E552E55282B46F
:101A10000FD0500EE66EC30EE66EE66AE66ACCDCC8
:101A2000E552E552E552E552040E0701A06FA16BA5
:101A30000701A13504E2A0510008000EA15505E2FE
:101A4000A0C7F3FFA1C7F4FF23D082B61CD0500E6D
:101A5000E66EC30EE66EE66AE66AAEDCE552E55275
:101A6000E552E55282B60FD0500EE66EC30EE66E1A
:101A7000E66AE66AA1DCE552E552E552E552050E5A
:101A80000701A06FA16BA0C7F3FFA1C7F4FF00D0AF
:101A9000120007018AAF05D0010EE66EE1EC00F0FE
:101AA000E552010EE66EE66AC8EC03F0E552E55237
:101AB0000701146B156B000E145D010E155946E2FB
:101AC000240E1425F66E400E1521F76E0800F5CF92
:101AD00018F018C009F09AEC1CF007C014F008C008
:101AE00015F009C016F00AC017F00C6A0D6A0E6AEC
:101AF000410E0F6E14C007F015C008F016C009F0B3
:101B000017C00AF072EC1DF007C074F708C075F733
:101B100009C076F70AC077F774C707F075C708F0F1
:101B200076C709F077C70AF058EC1EF00950E66E48
:101B3000000E07011425E96E060E1521EA6EE55226
:101B4000E750EF6E142B000E1523B5D712000701D6
:101B50008AAF05D0010EE66EE1EC00F0E552020E10
:101B6000E66EE66AC8EC03F0E552E5520701146B35
:101B7000156B800E145D000E15590CE2000E142535
:101B8000E96E060E1521EA6E1F0EEF6E142B000E85
:101B90001523EFD7800E146F156B000E145D010E28
:101BA00015590BE2000E1425E96E060E1521EA6E9A
:101BB000EF6A142B000E1523F0D7120007018AAF2D
:101BC00005D0010EE66EE1EC00F0E552030EE66E84
:101BD000E66AC8EC03F0E552E5520701146B156B99
:101BE000800E145D000E155940E214C708F015C7A9
:101BF00009F0ABEC1CF007C014F008C015F009C0E8
:101C000016F00AC017F00C6A0D6A800E0E6E400EB8
:101C10000F6E14C007F015C008F016C009F017C009
:101C20000AF072EC1DF007C074F708C075F709C020
:101C300076F70AC077F774C707F075C708F076C75C
:101C400009F077C70AF058EC1EF00950E66E000E56
:101C500007011425E96E060E1521EA6EE552E750DC
:101C6000EF6E142B000E1523BBD7800E146F156B6F
:101C7000000E145D010E155949E214C718F015C77E
:101C800019F0FF0ED8801856000E195618C008F02B
:101C900019C009F0ABEC1CF007C014F008C015F037
:101CA00009C016F00AC017F00C6A0D6A800E0E6E9D
:101CB000400E0F6E14C007F015C008F016C009F0F2
:101CC00017C00AF072EC1DF007C074F708C075F772
:101CD00009C076F70AC077F774C707F075C708F030
:101CE00076C709F077C70AF058EC1EF00950E66E87
:101CF000000E07011425E96E060E1521EA6EE55265
:101D0000E750EF6E142B000E1523B2D71200070117
:101D10008AAF05D0010EE66EE1EC00F0E552040E4C
:101D2000E66EE66AC8EC03F0E552E5520701146B73
:101D3000156B000E145D010E15593FE214C708F033
:101D400015C709F0ABEC1CF007C014F008C015F083
:101D500009C016F00AC017F00C6A0D6A0E6A410E2F
:101D60000F6E14C007F015C008F016C009F017C0B8
:101D70000AF072EC1DF007C074F708C075F709C0CF
:101D800076F70AC077F774C707F075C708F076C70B
:101D900009F077C70AF058EC1EF00950E66E000E05
:101DA00007011425E96E060E1521EA6EE552E7508B
:101DB000EF6E142B000E1523BCD7120007018AAF5B
:101DC00005D0010EE66EE1EC00F0E552050EE66E80
:101DD000E66AC8EC03F0E552E5520701146B156B97
:101DE000000E145D010E155948E214C718F015C70E
:101DF00019F0FF0ED8801856000E195618C008F0BA
:101E000019C009F0ABEC1CF007C014F008C015F0C5
:101E100009C016F00AC017F00C6A0D6A0E6A410E6E
:101E20000F6E14C007F015C008F016C009F017C0F7
:101E30000AF072EC1DF007C074F708C075F709C00E
:101E400076F70AC077F774C707F075C708F076C74A
:101E500009F077C70AF058EC1EF00950E66E000E44
:101E600007011425E96E060E1521EA6EE552E750CA
:101E7000EF6E142B000E1523B3D7120007018AAFA3
:101E800005D0010EE66EE1EC00F0E552060EE66EBE
:101E9000E66AC8EC03F0E552E5520701000ED8806F
:101EA0002255000E23552CE2FF0E225D000E235911
:101EB00027E2146B156B2251145D235115590CE266
:101EC000000E1425E96E060E1521EA6E1F0EEF6E48
:101ED000142B000E1523EFD722C714F723C715F7CD
:101EE000000E145D010E15590BE2000E1425E96E6B
:101EF000060E1521EA6EEF6A142B000E1523F0D79B
:101F00001200F29807018A8F010EE66EE1EC00F0F4
:101F1000E55278C7E6FF79C7E6FFC8EC03F0E55263
:101F2000E552BDDCF3CF16F7F4CF17F70701000E2B
:101F3000D8801655000E175501E3BAD30B0E165D67
:101F4000000E175901E3B4D3030E165D000E1759A6
:101F500001E34FD10A0E781901E1795101E12ED147
:101F6000090E781901E1795101E1FBD0080E7819C9
:101F700001E1795101E1EDD0070E781901E17951C4
:101F800001E17FD0060E781901E179516AE0050E72
:101F9000781901E1795155E0040E781901E1795180
:101FA00040E0030E781901E179512BE0020E781917
:101FB00001E1795116E0010E781901E1795101E052
:101FC00018D167DDF1C1E6FFF2C1E6FFF3C1E6FF1C
:101FD000F4C1E6FF2BEC0BF0E552E552E552E55279
:101FE00008D1B5DDF1C1E6FFF2C1E6FFF3C1E6FFBE
:101FF000F4C1E6FF2BEC0BF0E552E552E552E55259
:10200000F8D0DCDDF1C1E6FFF2C1E6FFF3C1E6FF87
:10201000F4C1E6FF2BEC0BF0E552E552E552E55238
:10202000E8D075DEF1C1E6FFF2C1E6FFF3C1E6FFDD
:10203000F4C1E6FF2BEC0BF0E552E552E552E55218
:10204000D8D0BCDEF1C1E6FFF2C1E6FFF3C1E6FF86
:10205000F4C1E6FF2BEC0BF0E552E552E552E552F8
:10206000C8D00CDFF1C1E6FFF2C1E6FFF3C1E6FF25
:10207000F4C1E6FF2BEC0BF0E552E552E552E552D8
:10208000B8D0020EE66EE1EC00F0E552060EE66E08
:10209000020EE66EC4EC00F0E552E55222C708F0ED
:1020A00023C709F0ABEC1CF007C018F008C019F00A
:1020B00009C01AF00AC01BF00C6A0D6AC80E0E6E39
:1020C000420E0F6E18C007F019C008F01AC009F0D0
:1020D0001BC00AF0C5EC1DF007C014F008C015F0D5
:1020E00009C016F00AC017F00C6A0D6A7F0E0E6E5A
:1020F000430E0F6E14C007F015C008F016C009F0AB
:1021000017C00AF072EC1DF007C070F708C071F735
:1021100009C072F70AC073F7020EE66EDEC1E6FF71
:10212000DFC1E6FF70C7E6FF71C7E6FF72C7E6FFD3
:1021300073C7E6FFD2EC04F0146E070EE15E145094
:10214000DEC1E6FFDFC1E6FFA3EC00F0E552E55299
:1021500050D0020EE66EE1EC00F0E552FDEC08F026
:1021600048D0010EE66EE1EC00F0E552090EE66E95
:10217000E66AC8EC03F0E552E55220C7E9FF21C743
:10218000EAFFD890E936EA361C0EE926010EEA226B
:10219000EECFF1F1EFCFF2F10101F36BF46BF1C18E
:1021A000E6FFF2C1E6FFF3C1E6FFF4C1E6FF2BEC68
:1021B0000BF0E552E552E552E5521BD0010EE66EFA
:1021C000E1EC00F0E5520A0EE66EE66AC8EC03F0B8
:1021D000E552E552F1C1E6FFF2C1E6FFF3C1E6FFC9
:1021E000F4C1E6FF2BEC0BF0E552E552E552E55267
:1021F00000D00701040E161901E1175106E0050E83
:10220000161901E1175101E053D20A0E781901E1C4
:10221000795101E1B7D1090E781901E1795101E154
:1022200033D1080E781901E1795101E1DED0070EB2
:10223000781901E1795101E03BD2010EE66EE1EC43
:1022400000F0E552070EE66EE66AC8EC03F0E552D0
:10225000E552A00EE66E860EE66E010EE66EE66AAA
:10226000DCEC09F0E552E552E552E552020EE66E6D
:10227000E1EC00F0E5524FEC0CF0F3CF16F7F4CFA1
:1022800017F70701030E225D000E235902E2166BB9
:10229000176BFD0ED8802255000E235502E2166BF7
:1022A000176B040E161901E117510AE1222B000EDB
:1022B00023230D0EE66EE66AC8EC03F0E552E55204
:1022C0000701050E161901E117510AE12207000E58
:1022D000235B0E0EE66EE66AC8EC03F0E552E552AB
:1022E000060EE66E020EE66EC4EC00F0E552E55214
:1022F00022C708F023C709F0ABEC1CF007C018F0A8
:1023000008C019F009C01AF00AC01BF00C6A0D6A67
:10231000C80E0E6E420E0F6E18C007F019C008F0FE
:102320001AC009F01BC00AF0C5EC1DF007C014F07C
:1023300008C015F009C016F00AC017F00C6A0D6A43
:102340007F0E0E6E430E0F6E14C007F015C008F01E
:1023500016C009F017C00AF072EC1DF007C070F744
:1023600008C071F709C072F70AC073F7020EE66E73
:10237000DEC1E6FFDFC1E6FF70C7E6FF71C7E6FF1B
:1023800072C7E6FF73C7E6FFD2EC04F0146E070EC7
:10239000E15E1450DEC1E6FFDFC1E6FFA3EC00F012
:1023A000E552E5520701030E161901E1175101E04C
:1023B00062D7010EE66EE1EC00F0E552060EE66E25
:1023C000E66AC8EC03F0E552E55258DDF1C1E6FFDC
:1023D000F2C1E6FFF3C1E6FFF4C1E6FF2BEC0BF020
:1023E000E552E552E552E55263D1010EE66EE1ECAD
:1023F00000F0E552080EE66EE66AC8EC03F0E5521E
:10240000E552A00EE66E860EE66E010EE66EE66AF8
:10241000DCEC09F0E552E552E552E552020EE66EBB
:10242000E1EC00F0E5520701040E161901E1175125
:102430000CE1030E1BAF02D0D89003D01A5D000E42
:102440001B5903E21A2B000E1B23050E161901E17E
:1024500017510AE11B3504E21A510108000E1B5501
:1024600003E21A07000E1B5BFDEC08F0A00EE66EFF
:10247000860EE66E010EE66EE66ADCEC09F0E552C9
:10248000E552E552E55214D1010EE66EE1EC00F0A2
:10249000E552090EE66EE66AC8EC03F0E552E55235
:1024A000A00EE66E860EE66E010EE66EE66ADCECC7
:1024B00009F0E552E552E552E552020EE66EE1EC16
:1024C00000F0E5524FEC0CF0F3CF16F7F4CF17F70E
:1024D0000701040E161901E117510DE1202B000E22
:1024E0002123213504E220513F08000E215503E24B
:1024F000010E206F216B050E161901E117510FE136
:102500002007000E215B010E21AF02D0D89003D02E
:10251000205D000E215903E23F0E206F216B20C782
:10252000E9FF21C7EAFFD890E936EA361C0EE92612
:10253000010EEA22EECFF1F1EFCFF2F10101F36BE0
:10254000F46BF1C1E6FFF2C1E6FFF3C1E6FFF4C1AF
:10255000E6FF2BEC0BF0E552E552E552E552500E4A
:10256000E66EC30EE66EE66AE66ADCEC09F0E5525A
:10257000E552E552E5520701030E161901E1175124
:10258000A1E196D0010EE66EE1EC00F0E5520A0EF4
:10259000E66EE66AC8EC03F0E552E552A00EE66E80
:1025A000860EE66E010EE66EE66ADCEC09F0E55298
:1025B000E552E552E552020EE66EE1EC00F0E5521E
:1025C0004FEC0CF0F3CF16F7F4CF17F7D8900101CA
:1025D000F451000A08E6020EF15D000EF259000EF9
:1025E000F359000EF45903E20701166B176B010152
:1025F000F435000EF41909E6D8803F0EF1559C0E13
:10260000F255000EF355000EF45503E20701166B68
:10261000176B0701040E161901E117510DE10101B5
:10262000F12B000EF223F323F4230D0EE66EE66A7F
:10263000C8EC03F0E552E5520701050E161901E159
:1026400017510DE10101F107000EF25BF35BF45B42
:102650000E0EE66EE66AC8EC03F0E552E552060E91
:10266000E66E020EE66EC4EC00F0E552E552F1C1F2
:10267000E6FFF2C1E6FFF3C1E6FFF4C1E6FF2BEC93
:102680000BF0E552E552E552E552500EE66EC30EF0
:10269000E66EE66AE66ADCEC09F0E552E552E552E0
:1026A000E5520701030E161901E1175189E100D027
:1026B0000701030E161901E117511BE1010EE66E29
:1026C000E1EC00F0E55278C7E6FF79C7E6FFC8EC19
:1026D00003F0E552E552F1C1E6FFF2C1E6FFF3C1B6
:1026E000E6FFF4C1E6FF2BEC0BF0E552E552E552B4
:1026F000E5520701136B166B176B9E90F2889D8A4B
:102700008A9F1200980EE66E3A0EE66EE66AE66A58
:10271000DCEC09F0E552E552E552E55235EC0AF001
:1027200007010B6B0C6B829A600E046F000E056F35
:1027300004C702F705C703F701019E0EDE6F010E05
:10274000DF6F0701866B876B886B896B8B6B8B8D5B
:102750008B898B958B9B8B978B918B93116B126BCA
:102760000F6B106B926B936B8A9FB3EC01F00C0EA6
:10277000E66E33EC02F0E552400EE66E0D0EE66EAC
:10278000030EE66EE66ADCEC09F0E552E552E5522E
:10279000E55243EC02F0DEC1E6FFDFC1E6FFFCECF0
:1027A00001F0E552E552F3CF18F7F4CF19F743ECF7
:1027B00002F0828A02C114F003C115F0166A14C037
:1027C000E6FF15C0E6FF16C0E6FF9E0EE66E010EA0
:1027D000E66E61EC28F0176E050EE15E17509E0E56
:1027E000E66E010EE66EFCEC01F0E552E552F3CF29
:1027F00018F7F4CF19F743EC02F0100EE66E270E2F
:10280000E66EE66AE66ADCEC09F0E552E552E5526E
:10281000E5521AC114F01BC115F0166A14C0E6FF88
:1028200015C0E6FF16C0E6FF9E0EE66E010EE66ED0
:1028300061EC28F0176E050EE15E17509E0EE66EF5
:10284000010EE66EFCEC01F0E552E552F3CF18F70D
:10285000F4CF19F743EC02F016C114F017C115F0CC
:10286000166A14C0E6FF15C0E6FF16C0E6FF9E0E0E
:10287000E66E010EE66E61EC28F0176E050EE15E65
:1028800017509E0EE66E010EE66EFCEC01F0E5526E
:10289000E552F3CF18F7F4CF19F718C114F019C1A6
:1028A00015F0166A14C0E6FF15C0E6FF16C0E6FF75
:1028B0009E0EE66E010EE66E61EC28F0176E050EB8
:1028C000E15E17509E0EE66E010EE66EFCEC01F026
:1028D000E552E552F3CF18F7F4CF19F7000EE66E84
:1028E000E66AC8EC03F0E552E5520E0EE66EE66AC3
:1028F000C8EC03F0E552E5520F0EE66EE66AC8EC4E
:1029000003F0E552E55243EC02F014C114F015C196
:1029100015F0166A14C0E6FF15C0E6FF16C0E6FF04
:102920009E0EE66E010EE66E61EC28F0176E050E47
:10293000E15E17509E0EE66E010EE66EFCEC01F0B5
:10294000E552E552F3CF18F7F4CF19F7240EF66EDF
:10295000440EF76E0900F5CF6CF70900F5CF6DF75F
:102960000900F5CF6EF70800F5CF6FF7060EE66E9B
:10297000DEC1E6FFDFC1E6FF6CC7E6FF6DC7E6FF1D
:102980006EC7E6FF6FC7E6FFD2EC04F0146E070EC9
:10299000E15E1450DEC1E6FFDFC1E6FFFCEC01F0B2
:1029A000E552E552F3CF18F7F4CF19F743EC02F0F4
:1029B000829A07018A8F0EEC00F0A00EE66E860E5A
:1029C000E66E010EE66EE66ADCEC09F0E552E552D1
:1029D000E552E552E66A010EE66EC4EC00F0E552FF
:1029E000E552A00EE66E520EE66E80EC00F0E55267
:1029F000E552E66A020EE66EC4EC00F0E552E552DE
:102A0000000EE66EE66AC8EC03F0E552E5520701F7
:102A10008A9F800EE66E1A0EE66E060EE66EE66A77
:102A2000DCEC09F0E552E552E552E552020E0701F1
:102A30001A6F1B6B0D0EE66EE66AC8EC03F0E552EA
:102A4000E552FDEC08F049EC0AF00701906B916B40
:102A5000146B156B000E145D010E155946E2240E21
:102A60001425F66E400E1521F76E0800F5CF18F00C
:102A700018C009F09AEC1CF007C014F008C015F05B
:102A800009C016F00AC017F00C6A0D6A0E6A410EF2
:102A90000F6E14C007F015C008F016C009F017C07B
:102AA0000AF072EC1DF007C074F708C075F709C092
:102AB00076F70AC077F774C707F075C708F076C7CE
:102AC00009F077C70AF058EC1EF00950E66E000EC8
:102AD00007011425E96E060E1521EA6EE552E7504E
:102AE000EF6E142B000E1523B5D7010E786F796B9E
:102AF0000A0E206F216B0101E80EF16F030EF26FD9
:102B0000F36BF46B12C114F013C115F0166A14C004
:102B1000E6FF15C0E6FF16C0E6FF9E0EE66E010E4C
:102B2000E66E61EC28F0176E050EE15E17509E0E02
:102B3000E66E010EE66EFCEC01F0E552E552F3CFD5
:102B400018F7F4CF19F70701866B876B886B896BD1
:102B5000F1C106F0F2C107F0F3C108F0F4C109F0C9
:102B6000C2EC1CF007C068F708C069F709C06AF733
:102B70000AC06BF76CC70CF06DC70DF06EC70EF096
:102B80006FC70FF068C707F069C708F06AC709F098
:102B90006BC70AF072EC1DF007C064F708C065F758
:102BA00009C066F70AC067F764C7E6FF65C7E6FFB6
:102BB00066C7E6FF67C7E6FF51EC27F0E552E5522E
:102BC000E552E55206C014F007C015F008C016F033
:102BD00009C017F014C007F015C008F016C009F0BE
:102BE00017C00AF0AEEC1EF006C082F707C083F7EC
:102BF00008C084F709C085F79E0EE66E010EE66EEA
:102C000082C7E6FF83C7E6FF84C7E6FF85C7E6FF06
:102C100030EC24F0146E060EE15E14509E0EE66E4B
:102C2000010EE66EFCEC01F0E552E552F3CF18F729
:102C3000F4CF19F743EC02F0100EE66E270EE66EA5
:102C4000E66AE66ADCEC09F0E552E552E552E55247
:102C5000800E0701226F236B8A8F010EE66EE1EC76
:102C600000F0E552010EE66EE66AC8EC03F0E552AC
:102C7000E552020EE66EE1EC00F0E5529E0EE66EC5
:102C8000010EE66EA3EC00F0E552E552F1C1E6FF5D
:102C9000F2C1E6FFF3C1E6FFF4C1E6FF2BEC0BF057
:102CA000E552E552E552E55207018A9F800EE66E35
:102CB0001A0EE66E060EE66EE66ADCEC09F0E552E8
:102CC000E552E552E552828AD08ED09CD66A000E3B
:102CD000E66EE66AC3EC28F0E552E552840ED56E46
:102CE000F29AF298D09E9D6A9D8AA06AA36AAB88E8
:102CF0009D8AF28CF28EF28C07018A9F8E6B8F6B0D
:102D0000136B07010451021902E10551031902E195
:102D100082EF1BF04CEC02F00701076F8E2B000EC8
:102D20008F238A9F0751580A02E193EF1AF0020A93
:102D300001E1EED3080A01E1E3D3160A01E1D8D399
:102D4000100A01E1CDD3170A01E1C2D3100A01E153
:102D5000B7D3120A01E19AD3110A02E082EF1BF005
:102D60000A0EE66EE66AC8EC03F0E552E552010E83
:102D7000E66EE66A57EC0AF0E552E552F3CF1CF72F
:102D8000F4CF1DF70701200ED8801C55020E1D55EB
:102D90000AE3E00E1C5D010E1D5905E38B9B898A39
:102DA0008986899853D389888B8B200ED8801C55AF
:102DB000020E1D5501E37ED1899A8986200ED880A6
:102DC0001C55020E1D5513E2D8900101F451000A62
:102DD00008E65E0EF15DEA0EF259000EF359000EA0
:102DE000F45905E2F12B000EF223F323F42307013B
:102DF000400ED8801C55020E1D5514E2D8900101DA
:102E0000F451000A08E65E0EF15DEA0EF259000E7A
:102E1000F359000EF45906E2020EF127000EF223D8
:102E2000F323F4230701600ED8801C55020E1D55B4
:102E300014E2D8900101F451000A08E65D0EF15D3C
:102E4000EA0EF259000EF359000EF45906E2030E91
:102E5000F127000EF223F323F4230701800ED8801C
:102E60001C55020E1D5514E2D8900101F451000AC0
:102E700008E65B0EF15DEA0EF259000EF359000E02
:102E8000F45906E2050EF127000EF223F323F42392
:102E90000701A00ED8801C55020E1D5514E2D890D3
:102EA0000101F451000A08E6560EF15DEA0EF259EE
:102EB000000EF359000EF45906E20A0EF127000E37
:102EC000F223F323F4230701C00ED8801C55020E11
:102ED0001D5514E2D8900101F451000A08E6510E84
:102EE000F15DEA0EF259000EF359000EF45906E2B4
:102EF0000F0EF127000EF223F323F4230701E00E57
:102F0000D8801C55020E1D5514E2D8900101F451D1
:102F1000000A08E6470EF15DEA0EF259000EF35979
:102F2000000EF45906E2190EF127000EF223F323E6
:102F3000F4230701000ED8801C55030E1D5514E222
:102F4000D8900101F451000A08E6150EF15DEA0E71
:102F5000F259000EF359000EF45906E24B0EF12718
:102F6000000EF223F323F4230701200ED8801C5512
:102F7000030E1D5514E2D8900101F451000A08E631
:102F8000FC0EF15DE90EF259000EF359000EF459F2
:102F900006E2640EF127000EF223F323F423070167
:102FA000400ED8801C55030E1D5514E2D890010127
:102FB000F451000A08E6F70EF15DE90EF259000E31
:102FC000F359000EF45906E2C80EF127000EF22361
:102FD000F323F4230701600ED8801C55030E1D5502
:102FE00015E2D8900101F451000A08E6930EF15D54
:102FF000E90EF259000EF359000EF45907E22C0EB7
:10300000F127010EF223000EF323F4230701800EB3
:10301000D8801C55030E1D5515E2D8900101F451BE
:10302000000A08E6D00EF15DE80EF259000EF359E1
:10303000000EF45907E2900EF127010EF223000E64
:10304000F323F4230701A00ED8801C55030E1D5551
:1030500015E2D8900101F451000A08E66C0EF15D0A
:10306000E80EF259000EF359000EF45907E2F40E7F
:10307000F127010EF223000EF323F4230701C00E03
:10308000D8801C55030E1D5515E2D8900101F4514E
:10309000000A08E6780EF15DE60EF259000EF359CB
:1030A000000EF45907E2E80EF127030EF223000E9A
:1030B000F323F4230701E00E1C5D010E1D5901E30B
:1030C0007ED1898A8996E00E1C5D010E1D5914E29D
:1030D0000101F435000EF41909E6D880010EF1550E
:1030E000000EF255000EF355000EF45505E2F107FF
:1030F000000EF25BF35BF45B0701C00E1C5D010E7A
:103100001D5915E20101F435000EF41909E6D880C5
:10311000020EF155000EF255000EF355000EF45557
:1031200006E2020EF15F000EF25BF35BF45B070157
:10313000A00E1C5D010E1D5915E20101F435000EB3
:10314000F41909E6D880030EF155000EF255000E71
:10315000F355000EF45506E2030EF15F000EF25B2C
:10316000F35BF45B0701800E1C5D010E1D5915E237
:103170000101F435000EF41909E6D880050EF15569
:10318000000EF255000EF355000EF45506E2050E42
:10319000F15F000EF25BF35BF45B0701600E1C5DF8
:1031A000010E1D5915E20101F435000EF41909E66E
:1031B000D8800A0EF155000EF255000EF355000EA0
:1031C000F45506E20A0EF15F000EF25BF35BF45B6E
:1031D0000701400E1C5D010E1D5915E20101F43579
:1031E000000EF41909E6D8800F0EF155000EF255C5
:1031F000000EF355000EF45506E20F0EF15F000EBF
:10320000F25BF35BF45B0701200E1C5D010E1D59A0
:1032100015E20101F435000EF41909E6D880190E03
:10322000F155000EF255000EF355000EF45506E26E
:10323000190EF15F000EF25BF35BF45B0701000E09
:103240001C5D010E1D5915E20101F435000EF41943
:1032500009E6D8804B0EF155000EF255000EF355DD
:10326000000EF45506E24B0EF15F000EF25BF35BCD
:10327000F45B0701E00E1C5D000E1D5915E2010113
:10328000F435000EF41909E6D880640EF155000EED
:10329000F255000EF355000EF45506E2640EF15F90
:1032A000000EF25BF35BF45B0701C00E1C5D000EC9
:1032B0001D5915E20101F435000EF41909E6D88014
:1032C000C80EF155000EF255000EF355000EF455E0
:1032D00006E2C80EF15F000EF25BF35BF45B0701E0
:1032E000A00E1C5D000E1D5916E20101F435000E02
:1032F000F41909E6D8802C0EF155010EF255000E96
:10330000F355000EF45507E22C0EF15F010EF25B4F
:10331000000EF35BF45B0701800E1C5D000E1D596F
:1033200016E20101F435000EF41909E6D880900E7A
:10333000F155010EF255000EF355000EF45507E25B
:10334000900EF15F010EF25B000EF35BF45B070180
:10335000600E1C5D000E1D5916E20101F435000ED1
:10336000F41909E6D880F40EF155010EF255000E5D
:10337000F355000EF45507E2F40EF15F010EF25B17
:10338000000EF35BF45B0701400E1C5D000E1D593F
:1033900016E20101F435000EF41909E6D880E80EB2
:1033A000F155030EF255000EF355000EF45507E2E9
:1033B000E80EF15F030EF25B000EF35BF45B0701B6
:1033C0008BAB37D0DEC1E6FFDFC1E6FF1CC7E6FFEF
:1033D0001DC7E6FF96EC23F0E552E552E552E552B3
:1033E0004D0EE66E33EC02F0E5523D0EE66E33EC28
:1033F00002F0E552DEC1E6FFDFC1E6FFFCEC01F0C2
:10340000E552E552F3CF18F7F4CF19F7090EE66E3F
:1034100033EC02F0E552F1C1E6FFF2C1E6FFF3C181
:10342000E6FFF4C1E6FF2BEC0BF0E552E552E55266
:10343000E552F00EE66E490EE66E020EE66EE66AA4
:10344000DCEC09F0E552E552E552E5520701045182
:10345000021902E10551031904E04CEC02F00701E6
:10346000076F1B0E075D01E082D4F1C1E6FFF2C1D8
:10347000E6FFF3C1E6FFF4C1E6FF2BEC0BF0E552EB
:10348000E552E552E55241EC0CF03CD1080EE66EF7
:10349000E66AC8EC03F0E552E55207011A2B000E6C
:1034A0001B231B3504E21A510308000E1B5503E2CF
:1034B000010E1A6F1B6BFDEC08F041EC0CF022D1F1
:1034C000010E786F796B49EC0DF041EC0CF01AD1DC
:1034D000020E786F796BA7EC0DF041EC0CF012D175
:1034E000030E786F796BDEEC0DF041EC0CF00AD135
:1034F000040E786F796B87EC0EF041EC0CF002D182
:10350000050E786F796BDEEC0EF041EC0CF0FAD022
:103510000B510C1102E0000E01D0010E0B6F0C6B71
:1035200041EC0CF0EFD0060E786F796B070EE66E6B
:10353000E66AC8EC03F0E552E552010EC26E0A0ECF
:10354000E66E3CEC29F0E5525EEC29F059EC29F0EE
:10355000000901E0FBD747EC29F0F3CF22F7F4CFC5
:1035600023F722C708F023C709F0ABEC1CF007C013
:1035700018F008C019F009C01AF00AC01BF00C6A54
:103580000D6AC80E0E6E420E0F6E18C007F019C0FD
:1035900008F01AC009F01BC00AF0C5EC1DF007C006
:1035A00014F008C015F009C016F00AC017F00C6A34
:1035B0000D6A800E0E6E440E0F6E14C007F015C01B
:1035C00008F016C009F017C00AF072EC1DF007C031
:1035D00070F708C071F709C072F70AC073F70701E6
:1035E000D89023332233D89023332233000ED8804F
:1035F0002255000E235501E382D0FF0E225D000EFE
:10360000235901E37CD0146B156B2251145D2351B7
:1036100015590CE2000E1425E96E060E1521EA6E0E
:103620001F0EEF6E142B000E1523EFD722C714F7D1
:1036300023C715F7000E145D010E15590BE2000E9D
:103640001425E96E060E1521EA6EEF6A142B000EA2
:103650001523F0D7DEC1E6FFDFC1E6FF22C7E6FF94
:1036600023C7E6FF96EC23F0E552E552E552E5521A
:103670004D0EE66E33EC02F0E552300E07011625D2
:10368000E66E33EC02F0E5523D0EE66E33EC02F0EE
:10369000E552DEC1E6FFDFC1E6FFFCEC01F0E552DA
:1036A000E552F3CF18F7F4CF19F7090EE66E33ECB5
:1036B00002F0E552020EE66EDEC1E6FFDFC1E6FF74
:1036C00070C7E6FF71C7E6FF72C7E6FF73C7E6FF84
:1036D000D2EC04F0146E070EE15E1450DEC1E6FF7A
:1036E000DFC1E6FFFCEC01F0E552E552F3CF18F73D
:1036F000F4CF19F7250EE66E33EC02F0E55241ECFB
:103700000CF000D00701050ED8808E55000E8F55A5
:1037100001E391D00D0E075D01E08DD0906B916BB0
:10372000146B156B050E145D000E155918E2600E32
:103730001425E96E000E1521EA6EEF50E66EE66A7A
:103740000CEC29F0E552E55207019051F324906FFB
:103750009151F420916F142B000E1523E3D7050E21
:10376000901901E191512FE010C114F011C115F031
:10377000166A14C0E6FF15C0E6FF16C0E6FF9E0EEF
:10378000E66E010EE66E61EC28F0176E050EE15E46
:1037900017509E0EE66E010EE66EFCEC01F0E5524F
:1037A000E552F3CF18F7F4CF19F7829A200EE66EA0
:1037B0004E0EE66EE66AE66ADCEC09F0E552E5528A
:1037C000E552E55231D0826B836B846B856B0001CF
:1037D000656B600EE66E000EE66EEBEC22F0E552D5
:1037E000E55206C0F1F107C0F2F108C0F3F109C0DB
:1037F000F4F1F1C1E6FFF2C1E6FFF3C1E6FFF4C167
:10380000E6FF2BEC0BF0E552E552E552E552A00E37
:10381000E66E860EE66E010EE66EE66ADCEC09F0F8
:10382000E552E552E552E552828A41EC0CF0090E70
:103830000701786F796B123504E211510008000E10
:10384000125507E3103504E20F510008000E105521
:1038500025E200C1E6FF01C1E6FFC3EC01F0E5523D
:10386000E552F3CF0DF7F4CF0EF711C7E6FF12C7FD
:10387000E6FF62EC04F0E552E552090EE66E33EC29
:1038800002F0E5520FC7E6FF10C7E6FF62EC04F056
:10389000E552E552829A41EC0CF001D0828A070190
:1038A0008A8F010EE66EE1EC00F0E55278C7E6FF84
:1038B00079C7E6FFC8EC03F0E552E552A00EE66ECC
:1038C000860EE66E010EE66EE66ADCEC09F0E55265
:1038D000E552E552E55207018A9F9E90F288166BE9
:1038E000176B8851EA6A000FE96E060EEA22EFCFE5
:1038F00040FF820EE96E070EEA6E8651EE24866F57
:103900008751EE20876F8851EE20886F8951EE2015
:10391000896F1351E6E0C40EE66E090EE66EE66AA4
:10392000E66ADCEC09F0E552E552E552E55281EF3A
:1039300016F01200019E05D0019E09AE02D0096C5E
:10394000018E09C003F0026A136A126A860E046EC1
:10395000056A68EF1FF0019E08D0019E09AE05D0F0
:10396000086C091EE86A0922018E09C003F008C02C
:1039700002F0136A126A8E0E046E056A68EF1FF079
:10398000019E0CD0019E09AE09D0066C071E081ED0
:10399000091EE86A072208220922018E09C003F0E5
:1039A00008C002F007C013F006C012F09E0E046EAD
:1039B000056A68EF1FF00F7E016AA4EC1FF0BCECF3
:1039C0001FF001B64CEF1FF001A20AD001AA03D0EC
:1039D00001BE4CEF1FF001A458EF1FF055EF1FF090
:1039E00001AA05D001AC58EF1FF055EF1FF001A060
:1039F0000AD001A808D001BE04D001A402D061EF12
:103A00001FF065EF1FF0126A056A0F500A5C116E15
:103A100010E307C013F008C002F009C003F00AC0A9
:103A200010F00CC007F00DC008F00EC009F0013A0C
:103A300009D00CC013F00DC002F00EC003F00FC08F
:103A400010F0116C019E01BC018E10C004F001B099
:103A500094EF1FF01A0E116094EF1FF0046A0A6AC7
:103A600001A408D0076C081E091E0A1EE86A082275
:103A700009220A2201AC08D0136C021E031E041E88
:103A8000E86A022203220422066A115207E00A347D
:103A90000932083207320632112EF9D707501326A1
:103AA00008500222095003220A50042206C012F0D4
:103AB000019E04AE0BD0126C131E021E031E041EC8
:103AC000E86A1322022203220422018E04A006D0F7
:103AD000D8800332023213321232102A10C004F09E
:103AE00068EF1FF0016AA4EC1FF0BCEC1FF001B6F8
:103AF0004CEF1FF001A205D001BA4CEF1FF053EFBD
:103B00001FF001BA5FEF1FF001A005D001B84CEF24
:103B10001FF05FEF1FF001B853EF1FF0056A7F0E33
:103B20000A24046EE86A05220F50045EE86A055A0A
:103B30001A0E106E0A6A126A136A026A036A0C503D
:103B4000075E0D50085A0E50095A000E0A5A09E72E
:103B50000C5007260D5008220E500922000E0A2292
:103B600001D0128AD8900736083609360A36D8901E
:103B70001236133602360336102EE1D709500810DC
:103B80000710D8A4128A68EF1FF0016AA4EC1FF096
:103B9000BCEC1FF001B64CEF1FF001A205D001B83C
:103BA0004CEF1FF053EF1FF001AA05D001B04CEF0E
:103BB0001FF053EF1FF001B002D001A802D05FEF59
:103BC0001FF0056A0F500A24046EE86A05227E0E73
:103BD000045EE86A055A126A136A026A036A0E50A2
:103BE0000902F4CF03F0F3CF02F00D500902F350B5
:103BF0001326F4500222000E03220E500802F35046
:103C00001326F4500222000E03220C500902F35036
:103C10001226F4501322000E022203220D50080235
:103C2000F3501226F4501322000E022203220E50EB
:103C30000702F3501226F4501322000E0222032230
:103C40000C500802F4501226000E13220222032206
:103C50000D500702F4501226000E132202220322F6
:103C600068EF1FF0006A0EAE3BEF1EF00D6C0E1EEB
:103C7000E86A0E22001E09AE43EF1EF0086C091E12
:103C8000E86A0922001EF6EC28F009BE53EF1EF088
:103C900000AE000C086C091EE86A0922046C051EBF
:103CA000E86A0522000C00BE4AEF1EF00188FF0CF6
:103CB000016AA4EC1FF001B662EF1EF001A20AD067
:103CC00001B403D07F0E096E19D0800E096E16D094
:103CD000096A14D001B0FCD7870E0A60F1D77E0EB6
:103CE0000A64F6D7860E0A5C04E0D89009320A2AE4
:103CF000F9D701A403D0096C09AEEAD71200016A12
:103D0000A4EC1FF001B689EF1EF001A20ED001B4A1
:103D100005D07F0E096EFF0E086E1FD0800E096E53
:103D2000086A1BD0096A086A18D001B0FBD78F0E49
:103D30000A60EDD77E0E0A64F5D78E0E0A5C05E0A8
:103D4000D890093208320A2AF8D701A406D0086CA4
:103D5000091EE86A092209AEE5D71200016AA4EC3F
:103D60001FF001B6B8EF1EF001A20FD001B407D0CA
:103D70007F0E096EFF0E086E076E066E25D0800E50
:103D8000096E01D0096A000EF6D701B0FBD7066AAA
:103D90009F0E0A60EBD77E0E0A64F4D79E0E0A5C73
:103DA00007E0D89009320832073206320A2AF6D7DD
:103DB00001A40AD0066C071E081E091EE86A072225
:103DC0000822092209AEDED71200F7EC1EF001B678
:103DD000000C01B0000C01B4000C010CF7EC1EF05B
:103DE00001B6000C01B0000C01A4000C010C016A2A
:103DF000A4EC1FF0BCEC1FF001B6120001AE08D01D
:103E000001A004D001A802D001801200019012008C
:103E10000F500A5C0BE10E50095C08E10D50085C84
:103E200005E10C50075C02E101801200D8A002D02D
:103E3000018E10D00A500FC00AF00F6E09500EC04C
:103E400009F00E6E08500DC008F00D6E07500CC042
:103E500007F00C6E0F500A5C10E0FF0F09E00190B4
:103E600001B403D001AE0184120001AE019412002E
:103E70000F2AD8900E320D320C320C50075E0D50C6
:103E8000085A0E50095A09BEEAD7D89007360836A4
:103E900009360A2EF8D7C8D77F0E0A6EFF0E096EB4
:103EA000086E076E12007F0E01BEFF0E0A6E02D072
:103EB0007F0E0A6E800E096E086A076AF3D701AE9C
:103EC00004D0800E0A6E096AF7D70A6A096AF4D725
:103ED0000350021013101210F8E005BEF0D703BE15
:103EE0000CD004500510EBE0D89012361336023691
:103EF00003360406D8A00506F2D70550D4E10428FD
:103F0000D2E012AE11D07F0E121402E113A00CD039
:103F1000132AE86A0222032207E3D880033202321E
:103F20001332042A0428BFE00450C9E013C007F08C
:103F300002C008F00334096E04300A6E09320A9E8A
:103F400001BE0A8E52EF1FF009360A3602E30184E1
:103F5000017E06E101800A6A096A086A076A12009E
:103F60000A2803E0D88009321200D890093202E111
:103F700001821200018612000E360F3602E3018C18
:103F8000017E06E101880F6A0E6A0D6A0C6A120052
:103F90000F2803E0D8800E321200D8900E32EAE1EA
:103FA000018A1200008080808080800000C0C0C034
:103FB000C0C0C00000E0E0E0E0E0E00000F0F0F0B1
:103FC000F0F0F00000F8F8F8F8F8F80000FCFCFC5D
:103FD000FCFCFC0000FEFEFEFEFEFE0000FFFFFFFC
:103FE000FFFFFF000010181C1E1C18100001030723
:103FF0000F070301040E1F0E0E0E0E0E0E0E0E0EF8
:104000000E1F0E0402040E111F100E0008040E11E4
:104010001F100E0008040E010F110F000205020010
:1040200000000000808285888B8E9194979A9DA0D5
:10403000A2A5A8ABADB0B3B5B8BBBDC0C2C5C7C91A
:10404000CCCED0D2D4D6D8DADCDEE0E2E3E5E6E8C6
:10405000E9EBECEDEEEFF0F1F2F3F4F5F5F6F6F74F
:10406000F7F7F7F7F8F7F7F7F7F7F6F6F5F5F4F3EC
:10407000F2F1F0EFEEEDECEBE9E8E6E5E3E2E0DEAD
:10408000DCDAD8D6D4D2D0CECCC9C7C5C2C0BDBB6D
:10409000B8B5B3B0ADABA8A5A2A09D9A9794918EE8
:1040A0008B888582807D7A7774716E6B6865625FBC
:1040B0005D5A5754524F4C4A4744423F3D3A383676
:1040C00033312F2D2B29272523211F1D1C1A1917AA
:1040D0001614131211100F0E0D0C0B0A0A09090801
:1040E0000808080808080808080809090A0A0B0C43
:1040F0000D0E0F10111213141617191A1C1D1F2163
:10410000232527292B2D2F313336383A3D3F424482
:10411000474A4C4F5254575A5D5F6265686B6E71E7
:1041200074777A7D000102030405060708090A0B6B
:104130000C0D0E0F101112131415161718191A1B47
:104140001C1D1E1F202122232425262728292A2B37
:104150002C2D2E2F303132333435363738393A3B27
:104160003C3D3E3F404142434445464748494A4B17
:104170004C4D4E4F505152535455565758595A5B07
:104180005C5D5E5F606162636465666768696A6BF7
:104190006C6D6E6F707172737475767778797A7BE7
:1041A0007C7D7E7F808182838485868788898A8BD7
:1041B0008C8D8E8F909192939495969798999A9BC7
:1041C0009C9D9E9FA0A1A2A3A4A5A6A7A8A9AAABB7
:1041D000ACADAEAFB0B1B2B3B4B5B6B7B8B9BABBA7
:1041E000BCBDBEBFC0C1C2C3C4C5C6C7C8C9CACB97
:1041F000CCCDCECFD0D1D2D3D4D5D6D7D8D9DADB87
:10420000DCDDDEDFE0E1E2E3E4E5E6E7E8E9EAEB76
:10421000ECEDEEEFF0F1F2F3F4F5F6F7F8F9FAFB66
:10422000FCFDFEFFFFFFFFFFFFFFFFFFFFFFFFFFA4
:10423000FFFFFFFFFFFFFFFFFFFFFFFFFFFFFFFF8E
:10424000FFFFFFFFFFFFFFFFFFFFFFFFFFFFFFFF7E
:10425000FFFFFFFFFFFFFFFFFFFFFFFFFFFFFFFF6E
:10426000FFFFFFFFFFFFFFFFFFFFFFFFFFFFFFFF5E
:10427000FFFFFFFFFFFFFFFFFFFFFFFFFFFFFFFF4E
:10428000FFFFFFFFFFFFFFFFFFFFFFFFFFFFFFFF3E
:10429000FFFFFFFFFFFFFFFFFFFFFFFFFFFFFFFF2E
:1042A000FFFFFFFF00000000000000000000000012
:1042B00000000000000000000000000000000000FE
:1042C00000000000000000000000000000000000EE
:1042D00000000000000000000000000000000000DE
:1042E00000000000000000000000000000000000CE
:1042F00000000000000000000000000000000000BE
:1043000000000000000000000000000000000000AD
:10431000000000000000000000000000000000009D
:104320000000000008090B0D0F11131517181A1CB7
:104330001E2022242627292B2D2F31333536383ABB
:104340003C3E4042444547494B4D4F5153545658CB
:104350005A5C5E6062636567696B6D6F71727476DB
:10436000787A7C7E8081838587898B8D8F909294EB
:1043700096989A9C9E9FA1A3A5A7A9ABADAEB0B2FB
:10438000B4B6B8BABCBDBFC1C3C5C7C9CBCCCED00B
:10439000D2D4D6D8DADBDDDFE1E3E5E7E9EAECEE1B
:1043A000F0F2F4F6F8F6F4F2F0EEECEAE9E7E5E321
:1043B000E1DFDDDBDAD8D6D4D2D0CECCCBC9C7C5CD
:1043C000C3C1BFBDBCBAB8B6B4B2B0AEADABA9A79D
:1043D000A5A3A19F9E9C9A98969492908F8D8B896D
:1043E00087858381807E7C7A78767472716F6D6B3D
:1043F0006967656362605E5C5A58565453514F4D0D
:104400004B4947454442403E3C3A38363533312FDC
:104410002D2B2927262422201E1C1A1817151311AC
:104420000F0D0B094CD8B43C4672616D6520457286
:1044300072657572206574204F766572666C6F7751
:1044400020646574656374696F6E203A2000506F54
:10445000727420636F6D6D20333834303062647352
:10446000206F7576657274004D617271756572208A
:104470003225206475207369676E616C0045534373
:1044800020706F757220736F727469720D004361D2
:10449000707475726520546175782073757220414F
:1044A0004443302000536F72746965204E6F726D03
:1044B000616C6520646520507267006361722072D0
:1044C000656375203A00557361676520513D313051
:1044D0004D687A2078342028504C4C290D00204516
:1044E0007272657572205361697369652E2E2E2E66
:1044F0002E0D0020496E697420436F6E73467265FD
:104500007120314B687A09002046616374657572C9
:1045100020444453203D200020496E74657266613A
:10452000636520766961205465726D696E616C20E7
:1045300052533233322045542F4F55207669612033
:10454000436C6176696572203520746F75636865A8
:1045500073202B204C43440D002047616D6D652076
:104560006465203120612033302E303030487A208D
:1045700028757020746F2036304B687A290D0043FF
:1045800031383A2031384632364B32325F44445368
:104590005F3133303331365F41444335625F4C43E2
:1045A000445F52533233325F42505F5242305F4376
:1045B00031382E630D002E2E2E2E2E2E2E2E203133
:1045C0002E303234560020322E303438560020340B
:1045D0002E3039365600FF0EE3CFEAFFE552FF0ECC
:1045E000E3CFE9FFE552E66AE66AE66AE66AD9CF12
:1045F000E6FFDACFE6FFFA0EE124D96EFF0EE220E5
:10460000DA6EE66AE66AE66AE66AE66A200EEF5C59
:1046100006E0090EEF5C03E0EF6603D06BD0EE50CE
:10462000F5D72D0EEF5C03E1FF0EE32A03D02B0E2E
:10463000EF5C01E1EE502F0EEF6444D03A0EEF60D4
:1046400041D0D890F50EE336F60EE336F70EE3369A
:10465000F80EE336FB0EDECFE3FFFC0EDECFE3FF0A
:10466000FD0EDECFE3FFFE0EDDCFE3FFDD52DD52B8
:10467000D890F50EE336F60EE336F70EE336F80E75
:10468000E336D890F50EE336F60EE336F70EE33652
:10469000F80EE336FB0EE350DE26FC0EE350DE227E
:1046A000FD0EE350DE22FE0EE350DD22DD52DD5230
:1046B000300EEE5CDE26000EDE22DE22DD22DD5232
:1046C000DD52B9D7FF0EE3CFE8FFE85213E0F50E55
:1046D000E31EF60EE31EF70EE31EF80EE31EF50EC4
:1046E000E32A08E1F60EE32A05E1F70EE32A02E1E8
:1046F000F80EE32AE552E552E552E552E552D9CFEC
:10470000E9FFDACFEAFFEECF06F0EECF07F0EECF0B
:1047100008F0EFCF09F0FF0EE3CFDAFFE552FF0E0E
:10472000E3CFD9FFE552E552E5521200D9CFE6FFBB
:10473000DACFE6FFFA0EE3CFD9FFFB0EE3CFDAFFC5
:10474000FD0EE35209E72D0EDE6EFC0EE31EE32A9A
:10475000FD0ED8B4E306E31EE652E652E652FD0E25
:10476000E124E76EFF0EE220E46EE652F70EE3CF9F
:10477000E6FFF70EE3CFE6FF06EC24F0F90EE124A6
:10478000E96EFF0EE220EA6EF6EC23F00AE1F3ECAC
:1047900023F009E1F6EC23F008E1F3EC23F007E164
:1047A00008D001EC24F0FCEC23F001EC24F0FCEC4C
:1047B00023F001EC24F0DE6AF90EE126FF0EE2227E
:1047C000FF0EE3CFDAFFE552FF0EE3CFD9FFE5524C
:1047D000FC0EE124E96EFF0EE220EA6EEECFF3FF5D
:1047E000EFCFF4FF1200EF380F0B1200EF500F0B5A
:1047F00002E1EE52D8841200EF380F0B300FDE6E5C
:104800001200EE500F0B300FDE6E1200FC0EE3CFE5
:10481000E9FFFD0EE3CFEAFF100EE66EEE6AEE6AE8
:10482000EF6AD890FD0EE336FE0EE336ED36ED3638
:10483000EF36FF0EE30609E027EC24F0EE5227ECFA
:1048400024F0EE5227EC24F0EDD7E56E1200030EB3
:10485000EF24E8B6EF6E300EEF24E8BEEF6E000CEA
:10486000D9CFE6FFDACFE6FFF80EE3CFD9FFF90E96
:10487000E3CFDAFFE652E652E652E652E652FB0E8C
:10488000E124E76EFF0EE220E46EE652F30EE3CF82
:10489000E6FFF30EE3CFE6FFF30EE3CFE6FFF30E02
:1048A000E3CFE6FFB5EC24F0F50EE124E96EFF0E50
:1048B000E220EA6EA2EC24F019E1A5EC24F018E164
:1048C000A2EC24F017E1A5EC24F016E1A2EC24F010
:1048D00015E1A5EC24F014E1A2EC24F013E1A5EC21
:1048E00024F012E1A2EC24F011E112D0ABEC24F0A0
:1048F000B0EC24F0ABEC24F0B0EC24F0ABEC24F002
:10490000B0EC24F0ABEC24F0B0EC24F0ABEC24F0F1
:10491000B0EC24F0DE6AF50EE126FF0EE222FF0E77
:10492000E3CFDAFFE552FF0EE3CFD9FFE552FA0EEF
:10493000E124E96EFF0EE220EA6EEECFF3FFEFCF47
:10494000F4FF1200EF380F0B1200EF500F0B02E1D3
:10495000EE52D8841200EF380F0B300FDE6E1200CB
:10496000EE500F0B300FDE6E1200FA0EE3CFE9FFB0
:10497000FB0EE3CFEAFF200EE66EEE6AEE6AEE6A09
:10498000EE6AEF6AD890FB0EE336FC0EE336FD0EBE
:10499000E336FE0EE336ED36ED36ED36ED36EF3628
:1049A000FF0EE3060FE0E4EC24F0EE52E4EC24F01A
:1049B000EE52E4EC24F0EE52E4EC24F0EE52E4EC9F
:1049C00024F0E1D7E56E1200030EEF24E8B6EF6E97
:1049D000300EEF24E8BEEF6E000CD9CFE6FFDACF41
:1049E000E6FFE1CFD9FFE2CFDAFF130EE12402E3C5
:1049F000E168E652E16E0C0EDB6AD950FA0FE96EFF
:104A0000FF0EDA20EA6E080EEECFDBFF090EEECFC6
:104A1000DBFF0A0EEECFDBFF0B0EEECFDBFF1FD965
:104A2000D950080F17D9EECFE6FFEECFE6FFEECF55
:104A3000E6FFEFCFE6FF36EC26F0146E060EE15CE3
:104A400002E2E16AE552E16E1450DF6E020EDF5CB5
:104A500001E0BCD0050EDBCF16F0060EDBCF17F061
:104A6000F80EDB50165C146EF90EDB501758156EFD
:104A70007F0E145E000E155A0D0E14C0DBFF0E0ED5
:104A800015C0DBFF0D0E0E0EDBCF15F00001800E02
:104A900015140AE0010EF36E0C0EF3CFDBFF070EC8
:104AA000DB5001E098D09DD00D0EDBCF14F00E0E40
:104AB000DBCF15F0D890155004E6170E145C000EED
:104AC000155801E39ED0186819687F0E1A6E1B6A8C
:104AD0000D0EDB501F0B18C014F019C015F01AC0D2
:104AE00016F01BC017F007E0D890173216321532B7
:104AF0001432E806F9E10F0E14C0DBFF100E15C0EA
:104B0000DBFF110E16C0DBFF120E17C0DBFF0F0E0E
:104B1000DBCF14F0100EDBCF15F0110EDBCF16F04B
:104B2000120EDBCF17F0D950010F94D8EE501416A7
:104B3000EE501516EE501616EE50171614501510AE
:104B40001610171002E1000E01D0010EE76E0C0ED8
:104B5000E7CFDBFFDB5055E0186A196A800E1A6E4A
:104B60001B6A010E1C6E1D6A1E6A1F6AD9500F0F48
:104B700071D8EE501C26EE501D22EE501E22EE5033
:104B80001F221C50185C146E1D501958156E1E50B3
:104B90001A58166E1F501B58176ED950010F5AD84D
:104BA0001450EE161550EE161650EE161750EE165F
:104BB000D950080FE66E000EDA20E66E50D8C4EC2D
:104BC00026F0E552E552E552E5521BD0DF0419E12B
:104BD000070EDB5006E0146A156A166A800E176E1F
:104BE00004D0146A156A166A176A080E14C0DBFF2F
:104BF000090E15C0DBFF0A0E16C0DBFF0B0E17C037
:104C0000DBFFF60EDBCFE9FFF70EDBCFEAFF0C0E82
:104C1000DBCFEFFF080EDBCF14F0090EDBCF15F072
:104C20000A0EDBCF16F00B0EDBCF17F014C006F028
:104C300015C007F016C008F017C009F0130EE15CAC
:104C400002E2E16AE552E16EE552E5CFDAFFE7CF35
:104C5000D9FF1200E96E000EDA20EA6E1200D95078
:104C6000010FE66E000EDA20E66E1200D9CFE6FFE5
:104C7000DACFE6FFE1CFD9FFE2CFDAFFE6521468E0
:104C800015687F0E166E176AD950FA0FE96EFF0E7F
:104C9000DA20EA6EEE501416EE501516EE50161687
:104CA000EE5017166AD814C0EEFF15C0EEFF16C0FE
:104CB000EEFF17C0EEFFFD0EDB50800B02E0010E91
:104CC00001D0000EE66E59D8060EE926000EEA2243
:104CD000E552E750EF6EFC0EDBCF14F0FD0EDBCF9C
:104CE00015F0D89014361536FC0E14C0DBFFFD0EFF
:104CF00015C0DBFFDB50E66E40D8040EE926000E3F
:104D0000EA22E552E750EE6EED6AFD0EDB50146EBE
:104D1000156AFF0E141818E1155016E12ED8EECFC3
:104D200014F0EECF15F0EECF16F0EFCF17F01450D1
:104D300015101610171006E0210E0101F96FFA6B1D
:104D4000800E0BD0040E09D0FD0EDB5008E115D803
:104D5000EE6AEE6AEE6AEE6A010EDF6E06D0020EB1
:104D6000DF6E0BD8EE52EE52EE8EDF50E552E5527A
:104D7000E5CFDAFFE7CFD9FF1200F80EDBCFE9FF6E
:104D8000F90EDBCFEAFF1200D9CFE6FFDACFE6FF5C
:104D9000E1CFD9FFE2CFDAFF5BD8153411E214502E
:104DA000FE08000E15540CE276D805E06CD8800E93
:104DB000EE6EEE6847D067D8800EEE6E7F0E0ED096
:104DC00047D8D890155004E6010E145C000E155813
:104DD0000BE261D805E057D8EE6A800EEE6E32D055
:104DE00052D8EE6AEE6A2ED047D8EECF14F0EECF4E
:104DF00015F0EECF16F0EFCF17F032D814C0EEFF5B
:104E000015C0EEFF16C0EEFF17C0EEFF21D81450FC
:104E1000010B05E025D8020E3AD8EF8E04D020D839
:104E2000020E35D8EF9E14D8D8901532143218D807
:104E3000030E2DD814C0EFFF1AD804E011D8030ECA
:104E400026D8EF8EE552E5CFDAFFE7CFD9FF120083
:104E500013D8040E1CD8EECF14F0EFCF15F01200CB
:104E6000FA0EDBCFE9FFFB0EDBCFEAFF120004D81E
:104E7000060E0DD8EF501200FC0EDBCFE9FFFD0E41
:104E8000DBCFEAFF1200ECDFEE6AEE6A1200E926E1
:104E9000000EEA221200220E0101F96FFA6B37EFC1
:104EA00027F0D9CFE6FFDACFE6FFE1CFD9FFE2CF97
:104EB000DAFF060EE12402E3E168E652E16ED95022
:104EC000050FE66E000EDA20E66E000EE66EE66A6C
:104ED000D950FA0FE96EFF0EDA20EA6EEECFE6FF48
:104EE000EECFE6FFEECFE6FFEFCFE6FFEDEC24F0EE
:104EF000146E080EE15C02E2E16AE552E16E1450C4
:104F0000010E06C0DBFF020E07C0DBFF030E08C068
:104F1000DBFF040E09C0DBFF050EDB502AE0040EA8
:104F2000DB50800B26E1146A156A800E166E3F0E68
:104F3000176ED950010FE96E000EDA20EA6EEECF3F
:104F400007F0EECF08F0EECF09F0EFCF0AF014C073
:104F50000CF015C00DF016C00EF017C00FF0DCEC11
:104F60001CF00AC0EDFF09C0EDFF08C0EDFF07C04F
:104F7000EFFF010EDBCF14F0020EDBCF15F0030EB6
:104F8000DBCF16F0040EDBCF17F014C006F015C00F
:104F900007F016C008F017C009F0060EE15C02E247
:104FA000E16AE552E16EE552E5CFDAFFE7CFD9FFDE
:104FB00012000E0EF66E000EF76E000EF86E000177
:104FC0000900F550E56F0900F550E66F03E1E5676C
:104FD00001D03DD00900F550E06F0900F550E16FB8
:104FE0000900F550E26F09000900F550E96E09006B
:104FF000F550EA6E090009000900F550E36F090059
:10500000F550E46F09000900F6CFE7F0F7CFE8F0BC
:10501000F8CFE9F0E0C0F6FFE1C0F7FFE2C0F8FF2B
:105020000001E35302E1E45307E00900F550EE6E9E
:10503000E307F8E2E407F9D7E7C0F6FFE8C0F7FFB7
:10504000E9C0F8FF0001E507000EE65BBFD71200DC
:10505000D9CFE6FFDACFE6FFE1CFD9FFE2CFDAFF23
:10506000AC6AAB6AFD0EDBB0AC88DBA202D0AC8CC4
:10507000AB8CDBB4AC8EDBA602D0AB8801D0AB8AA4
:10508000DBB8AC84DBBAAB86DBAC02D09D8A01D046
:105090009D9ADBAE02D09D8801D09D98FB0EDB501F
:1050A000AF6EFC0EDBCF15F015C014F0156A14506E
:1050B000B06EAC8AAB8EE552E5CFDAFFE7CFD9FF11
:1050C0001200FB0EE3CFF6FFFC0EE3CFF7FFFD0E61
:1050D000E3CFF8FFFE0EE3CFE9FFFF0EE3CFEAFFD9
:1050E000E9CFF3FFEACFF4FF0900F5CFEFFFEE665B
:1050F000FBD71200FE0EE3CFE9FFFF0EE3CFEAFF7E
:10510000F36AF46AEE5203E0F34AF42AFBD7120082
:10511000D9CFE6FFDACFE6FFE1CFD9FFE2CFDAFF62
:10512000E652F20E0101FB17ABAC03D0FB91ABB022
:10513000FB81ABB4FB85ABB2FB87AE50DF6EDF50BB
:10514000E552E552E5CFDAFFE7CFD9FF1200D9CF1C
:10515000E6FFDACFE6FFE1CFD9FFE2CFDAFFE65292
:10516000E652FC0EDBCFDEFFDBCFDDFF010EDB50B6
:10517000CF6EDF50CE6EE552E552E552E5CFDAFF55
:10518000E7CFD9FF1200D9CFE6FFDACFE6FFE1CFB4
:10519000D9FFE2CFDAFFE652E652FC0EDBCFDEFFAC
:1051A000DBCFDDFF010EDB50D76EDF50D66EE55250
:1051B000E552E552E5CFDAFFE7CFD9FF1200D9CFAC
:1051C000E6FFDACFE6FFE1CFD9FFE2CFDAFFACAC02
:1051D00004D0AC900101FBB3AC80FD0EDB50AD6E92
:1051E000E552E5CFDAFFE7CFD9FF1200056A046A7E
:1051F000100EE76ED89008360936043605360D5085
:10520000045C0E50055805E30D50045E0E50055A1F
:10521000082AE72EF0D71200F36AF46AFF0EE124A1
:10522000E96EFF0EE220EA6EED6607D02F0EEF6406
:1052300004D03A0EEF6001D0F32A1200380EF36E5C
:1052400000EE00F00F0E01D81200EA6002D0EE6A04
:10525000FCD7F350E9601200EE6AFCD71EEE00F0B6
:105260002EEE00F0F86A019CD9EC27F003EC00F078
:1052700082EC13F0FBD71200FF0EE350E84E120051
:10528000000000D000D000D0E82EFAD71200C450A1
:10529000176E166AC3501610F36E17C0F4FF120093
:1052A00031384632364B3232204444532043313871
:1052B00000FFC250020B01E0010E1200C282120078
:1052C00028444E4468447D448E44A544BB44C644AF
:1052D000DE44F3440845184559457F450100020066
:1052E00005000A00140032006400C800F401EE0258
:1052F000E803E204DC05D606D007C409BE0AB80BF1
:10530000AC0DA00F941188137C1570176419581BED
:105310004C1D401F342128231C251027F82AE02E7D
:10532000C832B036983A803E68425046384A204EDD
:105330000852F055D859C05DA86190657869606DD4
:10534000487130751879007DE880D084B888A08CC9
:10535000889070945898409C04A6C8AF244050523E
:105360004F4A45543A2031384632364B32325F4448
:1053700044532E6D6370200D0000000000000000FB
:10538000000000000000000000000000000000001D
:1053900000000000000000000000000000009E016E
:1053A00031323334353637383930313233343500F1
:1053B000000000000000000000FFFFFFFFFFFFFFF4
:1053C000FFFFFFFFFFFFFFFFFFFFFFFFFFFFFFFFED
:1053D000FFFFFFFFFFFFFFFFFFFFFFFFFFFFFFFFDD
:1053E000FFFFFFFFFFFFFFFFFFFFFFFFFFFFFFFFCD
:1053F000FFFFFFFFFFFFFFFFFFFFFFFFFFFFFFFFBD
:0200000400F00A
:100000002031384632364B32322034304D687A2037
:10001000513D31304D687A20504C4C78340D000001
:100020002053696E7573202020202020202020205E
:10003000202020202020202020202020200D000013
:100040002043617272652020202020202020202063
:10005000202020202020202020202020200D0000F3
:1000600020547269616E676C65202020202020205A
:10007000202020202020202020202020200D0000D3
:100080002044656E742064652073636965202020B8
:10009000202020202020202020202020200D0000B3
:1000A00020526576657273652064656E74206465A0
:1000B000207363696520202020202020200D00006F
:1000C0002052656374616E676C65206628546175A3
:1000D000782920202020202020202020200D000012
:1000E000205265676C6167652054617578205265A0
:1000F0006374616E676C652028706F74290D000051
:10010000205265676C616765206D61786920736F47
:10011000727469652044414320566F6C740D000071
:100120002043686F6978204672657175656E6365F6
:10013000203A2031207061726D692031360D000047
:10014000205265676C6167652046696E204672655E
:100150007175656E6365202020202020200D000031
:10016000202020202020202020202020202020208F
:10017000202020202020202020202020200D0000D2
:10018000202020202020202020202020202020206F
:10019000202020202020202020202020200D0000B2
:1001A00020496E697420736F7274696520444143FD
:1001B000206D6178693A20322C303438560D0000B9
:1001C000204D504C4142204944452056382E383964
:1001D0002C4331382056332E34342E20200D00008D
:1001E0002056657273696F6E2031362F30332F3190
:1001F0003320207061756C666A756A6F200D00008F
:1002000056657273696F6E2031362F30332F31335C
:10021000202020202053494E5553202020202020EC
:100220002020202020436172726520202020202081
:100230002020202020547269616E676C6520202088
:100240002044656E74732064652053434945202023
:100250007265762044656E74206465205343494579
:100260002020202052656374616E676C6520202019
:100270005265676C65205441555820526563742E51
:100280005265676C65204D61786920416D706C69BD
:1002900043686F6978204672657120466978657396
:1002A0005265676C61672066696E2046726571757C
:1002B000202020202020202020202020202020203E
:1002C000202020202020202020202020202020202E
:1002D000203E3E20202020202020202020202020E2
:1002E000203C3C20202020202020202020202020D6
:1002F00020202020202020202020202020202020FE
:10030000FFFFFFFFFFFFFFFFFFFFFFFFFFFFFFFFFD
:10031000FFFFFFFFFFFFFFFFFFFFFFFFFFFFFFFFED
:10032000FFFFFFFFFFFFFFFFFFFFFFFFFFFFFFFFDD
:10033000FFFFFFFFFFFFFFFFFFFFFFFFFFFFFFFFCD
:10034000FFFFFFFFFFFFFFFFFFFFFFFFFFFFFFFFBD
:10035000FFFFFFFFFFFFFFFFFFFFFFFFFFFFFFFFAD
:10036000FFFFFFFFFFFFFFFFFFFFFFFFFFFFFFFF9D
:10037000FFFFFFFFFFFFFFFFFFFFFFFFFFFFFFFF8D
:10038000FFFFFFFFFFFFFFFFFFFFFFFFFFFFFFFF7D
:10039000FFFFFFFFFFFFFFFFFFFFFFFFFFFFFFFF6D
:1003A000FFFFFFFFFFFFFFFFFFFFFFFFFFFFFFFF5D
:1003B000FFFFFFFFFFFFFFFFFFFFFFFFFFFFFFFF4D
:1003C000FFFFFFFFFFFFFFFFFFFFFFFFFFFFFFFF3D
:1003D000FFFFFFFFFFFFFFFFFFFFFFFFFFFFFFFF2D
:1003E000FFFFFFFFFFFFFFFFFFFFFFFFFFFFFFFF1D
:1003F000FFFFFFFFFFFFFFFFFFFFFFFFFFFFFFFF0D
:020000040030CA
:0E0000000032193C009D84000FC00FE00F403D
:020000040020DA
:08000000FFFFFFFFFFFFFFFF00
:00000001FF
